:0200000270008C
:10800000807F0020398507006185070063850700B0
:108010006585070067850700698507000000000087
:108020000000000000000000000000006B85070059
:108030006D850700000000006F850700718507004F
:108040007385070073850700738507007385070034
:108050007385070073850700738507007385070024
:108060007385070073850700738507007385070014
:10807000738507007DC307007385070073850700BC
:108080007385070095C70700738507007385070090
:108090003DC4070073850700CDC107007385070045
:1080A00073850700738507007385070073850700D4
:1080B00073850700738507000000000000000000C2
:1080C00073850700738507007385070073850700B4
:1080D00073850700738507007385070000000000A3
:1080E0000000000000000000000000000000000090
:1080F0000000000000000000000000000000000080
:10810000000000000000000000000000000000006F
:10811000000000000000000000000000000000005F
:1084000010B5054C237833B9044B13B10448AFF3CE
:1084100000800123237010BD882C00200000000084
:1084200014D0070008B5034B1BB103490348AFF351
:10843000008008BD000000008C2C002014D0070034
:10844000154B002B08BF134B9D46A3F5803A002126
:108450008B460F461348144A121A00F063F80F4B6C
:10846000002B00D098470E4B002B00D098470020DF
:10847000002104000D000D48002802D00C48AFF385
:10848000008000F02BF82000290004F0E3F900F050
:1084900011F800BF00000800807F002000000000ED
:1084A00000000000882C0020B438002000000000EC
:1084B0000000000008B5074B044613B10021AFF3DC
:1084C0000080054B1868836A03B19847204600F086
:1084D00031F800BF0000000018CC070070B50D4D4A
:1084E0000D4C641BA4100026A64209D10B4D0C4C68
:1084F00004F086FB641BA4100026A64205D170BDC3
:1085000055F8043B98470136EEE755F8043B984789
:108510000136F2E7682C0020682C0020682C00202F
:108520006C2C002002440346934200D1704703F8AC
:10853000011BF9E7FEE700BF0649074A074B9B1AF4
:1085400003DD043BC858D050FBDC03F053FEFFF7BB
:1085500077FF000020D00700002C0020882C00208E
:10856000FEE7FEE7FEE7FEE7FEE7FEE7FEE7FEE7E3
:10857000FEE7FEE770B5EFF3108672B60D4A946819
:108580000123A4B993600C4B0C4DD3F88010294003
:108590001160C3F88050D3F8841051604FF0FF325F
:1085A000C3F88420047006B962B6002070BD037061
:1085B000F9E700BF7434002000E100E0FC06FFBCD6
:1085C0002DE9F04FC9B008AA01F1400514464B78D7
:1085D0000E781B0443EA0663CE7833438E78043169
:1085E00043EA06238D4244F8043BF0D11024916BFA
:1085F00016464FEAF14383EA714383EA9123716A95
:10860000366852F8045F31440B444FEAB54181EAC1
:10861000F51181EAD50101340B44402CD363E6D136
:10862000D0E914E30093836D0193C36D0293036E4D
:108630000393436E0493836E0593C36E0693DDE943
:10864000057BDDE9031CDDE901592B4B009E0793F7
:1086500074464FF00008079B53F8042B07934FEA2A
:10866000F12383EAB11383EA716A08AB53F8283027
:108670001A440AEB020327EA010A01EA0C028AEA19
:1086800002021A444FEA743A86EA05035A448AEA17
:10869000B40A06EA050B234083EA0B038AEAB45ABC
:1086A00008F101089A44B8F1400F02EB0903BB46F8
:1086B0005244A94619D172440265009A2244426587
:1086C000019A32448265029A2A44C265039A1A4486
:1086D000049B02660B444366059B63448366069BCA
:1086E0003B44C36649B0BDE8F08F674635468C46CB
:1086F000264619461446AEE744CE07002DE9F04F52
:1087000093B0CDE9002002A892F90020B1E8005E04
:1087100006B4AAFB09124FF00003EBFB69234FF0EC
:108720000004ECFB69344FF00005EEFB69454FF0A7
:108730000006EBFB6A63ECFB6A3449185241764150
:108740005B41A9FB09784FF0000949F1000918EBDA
:108750000108A0E88001AAFB0A78574158EB0608F7
:10876000A0E88001EEFB6A454FF0000A4AF1000ADA
:108770004FF00001ECFB6B14EEFB6B454FF0000279
:10878000EEFB6C255FEA59094941644152416D4154
:1087900049F10009EBFB6B3A1AEB010AA0E8080467
:1087A000ACFB0C6A66415AEB020AA0E84004AEFB3F
:1087B0000E6A6E415AEB090AA0E8400406BC052A7D
:1087C00000F0E680A0F11400A1F11401B1E8E0434B
:1087D000A5FB0E344FF00005E6FB6E454FF000069A
:1087E000E7FB6E564FF00007E8FB6E674FF000089E
:1087F000E9FB6E784FF00009DB1864416D4176416A
:108800007F4158EB080859F1000950F804CB13EBED
:108810000C0350F804CB54EB0C0450F804CB55EB8C
:108820000C0550F804CB56EB0C0650F804CB57EB74
:108830000C0758F1000859F10009A0F11400EEFBF3
:108840000E89A0E8F803062A00F0A280A0F1180023
:10885000A1F11801B1E8E047A5FB0E344FF0000587
:10886000E6FB6E454FF00006E7FB6E564FF0000743
:10887000E8FB6E674FF00008E9FB6E784FF00009E7
:10888000EAFB6E894FF0000ADB1864416D417641C6
:108890007F4158EB080859EB09095AF1000A50F8D2
:1088A00004CB13EB0C0350F804CB54EB0C0450F83E
:1088B00004CB55EB0C0550F804CB56EB0C0650F8E6
:1088C00004CB57EB0C0750F804CB58EB0C0859F1CC
:1088D00000095AF1000AA0F11800EEFB0E9AA0E878
:1088E000F807072A54D0A0F11C00A1F11C01B1E83F
:1088F000E04FA5FB0E344FF00005E6FB6E454FF050
:108900000006E7FB6E564FF00007E8FB6E674FF07E
:108910000008E9FB6E784FF00009EAFB6E894FF022
:10892000000AEBFB6E9A4FF0000BDB1864416D41BF
:1089300076417F4158EB080859EB09095AEB0A0ABE
:108940005BF1000B50F804CB13EB0C0350F804CB95
:1089500054EB0C0450F804CB55EB0C0550F804CB49
:1089600056EB0C0650F804CB57EB0C0750F804CB31
:1089700058EB0C0850F804CB59EB0C095AF1000ADB
:108980005BF1000BA0F11C00EEFB0EABA0E8F80FB2
:10899000009B0198D3F8AC3002A9984713B0BDE80A
:1089A000F08F00EB81010023884200D3704751F81B
:1089B000042D43EA52030B60D307F5E710B5013AE3
:1089C00052B2130601D5002010BD50F8224051F8D4
:1089D00022309C4205D802F1FF32F2D24FF0FF3034
:1089E000F2E70120F0E710B500235CB2A24200DC00
:1089F00010BD51F8234040F823400133F5E7013919
:108A000010B549B2041D0A06CBB204D4013954F89A
:108A10002120002AF7D001335BB273B103F1804209
:108A2000013A50F82220002022B9013B00EB431309
:108A300018B210BD52080130F6E71846F9E74A119E
:108A4000012350F8220001F01F0103FA01F1084050
:108A5000704710B500231A465CB2A14203DCB2FA9B
:108A600082F0400910BD50F8234001332243F3E760
:108A7000002310B51C465AB2914200DC10BD40F8EC
:108A800023400133F7E72DE9F04FA5B01D4604ABB5
:108A9000CDE902318146294610461746FFF7AFFF60
:108AA000C0EB851004B2002C2646B8BF04F11F06A7
:108AB000634246F3471603F01F0304F01F0814A88F
:108AC00058BFC3F100083146FFF7D2FFB8F1000FDD
:108AD00030B22DDD14AB002203EB8000C8F1200C76
:108AE00013469D4219D82FB27B00019314AB03EBC0
:108AF000870705F1FF3824AB012603EB8808002C1B
:108B000054DA24AB03EB86062A4656F8881C4846FE
:108B1000FFF769FF25B0BDE8F08F57F8236006FA2C
:108B200008F10A4340F8042B013326FA0CF2D8E787
:108B300014AB2A46394603EB8000FFF754FFD2E717
:108B40000FFA82FE5AF8883C53F82EB024AB03EBA0
:108B50008202013052F8403C0B44BBEB030334BFAC
:108B6000012200229B4518BF11465CF8882C42F870
:108B70002E30019B42B29A42E2DB731A5E422946D2
:108B800014A85E41FFF70DFF24AB03EB85032946D4
:108B900053F8402C58F8403C384643EAC273013C35
:108BA00048F8403C24B2FFF7FCFEA8E724AB0020C5
:108BB000C6F1010C014603EB860A03EB8C0CD8E7E7
:108BC0002DE9F04F08B4F8CA04B451F8042BA3FB04
:108BD000028940F8048B4FF0000AE4FB629A4FF0E0
:108BE000000BE5FB62AB4FF0000CE6FB62BC4FF004
:108BF000000EE7FB62CE51F8042B4FF00008E3FBB8
:108C0000628940F8048BE4FB629AE5FB62ABE6FB09
:108C100062BCE7FB62CE51F8042B4FF00008E3FB87
:108C2000628940F8048BE4FB629AE5FB62ABE6FBE9
:108C300062BCE7FB62CE51F8042B4FF00008E3FB67
:108C4000628940F8048BE4FB629AE5FB62ABE6FBC9
:108C500062BCE7FB62CE51F8042B4FF00008E3FB47
:108C6000628940F8048BE4FB629AE5FB62ABE6FBA9
:108C700062BCE7FB62CE40F8049B40F804AB40F8CE
:108C800004BB40F804CB40F804EB0CBC052B00F00F
:108C90001E810C68A0F11400A1F11401A2F11402CC
:108CA00052F804EB4FF0000550F8046BE4FB6E56ED
:108CB00052F804EB50F8047BE4FB6E6752F804EBC7
:108CC00050F8048BE4FB6E7852F804EB50F8049BE8
:108CD000E4FB6E8952F804EB50F804ABE4FB6E9AA7
:108CE000A0F1140052F8044B51F804EB4FF0000CC3
:108CF000E4FB6EC540F804CB51F804EBE4FB6E5680
:108D000040F8045B51F804EBE4FB6E6740F8046B39
:108D100051F804EBE4FB6E7840F8047B51F804EB67
:108D2000E4FB6E8940F8048B51F804EBE4FB6E9A87
:108D3000A0E80006062B00F0CA800C68A0F118001D
:108D4000A1F11801A2F1180252F804EB4FF000054E
:108D500050F8046BE4FB6E5652F804EB50F8047BB9
:108D6000E4FB6E6752F804EB50F8048BE4FB6E787A
:108D700052F804EB50F8049BE4FB6E8952F804EBC4
:108D800050F804ABE4FB6E9A52F804EB50F804BBC5
:108D9000E4FB6EABA0F1180052F8044B51F804EB61
:108DA0004FF0000CE4FB6EC540F804CB51F804EB27
:108DB000E4FB6E5640F8045B51F804EBE4FB6E678D
:108DC00040F8046B51F804EBE4FB6E7840F8047B48
:108DD00051F804EBE4FB6E8940F8048B51F804EB86
:108DE000E4FB6E9A40F8049B51F804EBE4FB6EAB95
:108DF000A0E8000C072B6AD008B40C68A0F11C0096
:108E0000A1F11C01A2F11C0252F804EB4FF0000585
:108E100050F8046BE4FB6E5652F804EB50F8047BF8
:108E2000E4FB6E6752F804EB50F8048BE4FB6E78B9
:108E300052F804EB50F8049BE4FB6E8952F804EB03
:108E400050F804ABE4FB6E9A52F804EB50F804BB04
:108E5000E4FB6EAB52F804EB50F804CBE4FB6EBCC1
:108E6000A0F11C0052F8044B51F804EB4FF0000342
:108E7000E4FB6E3540F8043B51F804EBE4FB6E561E
:108E800040F8045B51F804EBE4FB6E6740F8046BB8
:108E900051F804EBE4FB6E7840F8047B51F804EBE6
:108EA000E4FB6E8940F8048B51F804EBE4FB6E9A06
:108EB00040F8049B51F804EBE4FB6EAB40F804ABC4
:108EC00051F804EBE4FB6EBCA0E8001808BCBDE858
:108ED000F08F30B51C4691B0054693F900306846D6
:108EE000FFF76EFED4F8AC3069462846984711B0BB
:108EF00030BDF0B5154689B01C4607460E461A46E9
:108F000029466846FFF7FAFB23466A463946384643
:108F1000FFF7DFFF23462A4669466846FFF7D9FF79
:108F200023466A4631463046FFF7D3FF09B0F0BD0D
:108F3000C3F10803DB0070B50133002403A500BFB3
:108F40005B1920C940CAAD1B20C0184720C940CAC0
:108F5000B54120C020C940CAB54120C020C940CA7F
:108F6000B54120C020C940CAB54120C020C940CA6F
:108F7000B54120C020C940CAB54120C020C940CA5F
:108F8000B54120C06441B4FA84F0400970BD00BF0F
:108F9000C3F10803DB0070B50133002403A500BF53
:108FA0005B1920C940CAAD1920C0184720C940CA62
:108FB000754120C020C940CA754120C020C940CA9F
:108FC000754120C020C940CA754120C020C940CA8F
:108FD000754120C020C940CA754120C020C940CA7F
:108FE000754120C06441204670BD00BFF0B5082225
:108FF00089B00C460646FFF7F6FCCB6A03930B6B71
:1090000004934B6B05938B6B0693CB6B07930027F5
:1090100008236A4669466846CDE901770097FFF75D
:10902000B7FF082305466A4631463046FFF7B0FFD2
:10903000236B0393636B0493A36B0593E36B05446A
:10904000CDE906376A46082369466846FFF7A0FF60
:10905000082305446A4631463046FFF799FF236AE4
:109060000093636A0193A36A0293A36B0693E36B75
:109070000793054408236A4631463046CDE9047714
:109080000397FFF785FF636A0093A36AA26B0193BE
:10909000E36A02930492636BE26B0393CDE90523C9
:1090A000236A0793054408236A4631463046FFF792
:1090B0006FFFE36A0093236B0193636B0293236A50
:1090C0000693A36A0793054408236A46314630464F
:1090D000CDE904770397FFF72BFF236B0093636BB6
:1090E0000193A36B0293E36B0393636A0693E36AB2
:1090F00007932D1A08236A4631463046CDE9047796
:10910000FFF716FF636B0093A36B0193E36B02936E
:10911000236A0393636A0493A36ACDE90537236B3B
:1091200007932D1A08236A4631463046FFF700FFA1
:10913000A36B0093E36BCDE90137636A0393A36AE2
:109140000493E36ACDE90537636B07932D1A08236F
:109150006A4631463046FFF7EBFE2D1A0D4C0FD410
:1091600035B9082231462046FFF728FC01280FD0E8
:109170000823224631463046FFF7DAFE2D1AEFE784
:109180000823224631463046FFF702FF2D18F7D458
:1091900009B0F0BD5CCC070070B5036813F00105A1
:1091A0000646144605D013460A460146FFF7F0FE70
:1091B000054621463046FFF7F4FB45B104F18042F5
:1091C000013A56F8223043F0004346F8223070BD91
:1091D000F0B50F46A1B006461946384615461C465E
:1091E000FFF737FC20B13046FFF742FC21B0F0BD5D
:1091F000224639466846FFF7F6FB294608A8FFF7DE
:10920000F2FB10A82146FFF733FC012318A81093A6
:10921000FFF72EFC224608A96846FFF7CFFB28B9C6
:10922000224610A93046FFF7DEFBDFE7009BDA0796
:1092300009D421466846FFF7B4FB2246294610A808
:10924000FFF7AAFFE6E7089BDB0707D4214608A83B
:10925000FFF7A7FB2246294618A8F1E70028234676
:109260001CDD08AA69466846FFF762FE214668468B
:10927000FFF797FB224618A910A8FFF79FFB0028CD
:1092800005DA10A923462A460846FFF781FE10A9F1
:10929000234618AA0846FFF74BFECEE708A96A4600
:1092A0000846FFF745FE214608A8FFF77AFB22464D
:1092B00010A918A8FFF782FB002805DA18A9234691
:1092C0002A460846FFF764FE18A9234610AA084656
:1092D000FFF72EFEBEE770B59DF910401E462346EF
:1092E0000546FFF725FE38B1234632462946284673
:1092F000BDE87040FFF74CBE70BD2DE9F0438BB068
:109300001446129D15F9046B00961F468046894647
:109310002B460246214602A8FFF7DDFF02A9129A5A
:109320000846FFF7EBF9129B02AA41464046FFF7B9
:10933000D0FD129B02AA21462046FFF7CAFD2B460C
:109340004A46394638460096FFF7C5FF129A394615
:1093500002A8FFF7D3F902A92B4642460846009619
:10936000FFF7B9FF02A92B46224608460096FFF7F1
:10937000B2FF2B464246214620460096FFF7ABFF40
:10938000129B224649464846FFF7A3FD2B4602AAF8
:10939000414620460096FFF79EFF129B2246394623
:1093A0003846FFF796FD2B464A4639463846009622
:1093B000FFF791FF324602A92046FFF714FB0BB0DE
:1093C000BDE8F0832DE9F04FEBB09346749F059113
:1093D000B7F9022097F9004012F11F0148BF02F1CE
:1093E0003E0141F347120292013A4FEA82096AA90B
:1093F00012AE82460DF1280801EB0900002140F869
:10940000C01C46F8221048F8221097F90110304687
:109410000D460A46002A40F0268103EB4103002D49
:1094200040F0278121463046FFF713FB002840F02B
:1094300016814046FFF70DFB0490002840F00F8195
:1094400007F12403029A039331461846FFF7B6FA50
:10945000012840F00481029A03984146FFF7AEFAD2
:10946000012840F0FC8042AEDDE902323046FFF7D1
:10947000AFFE6AAB9944B7F9023049F8605C13F16A
:109480001F0548BF03F13E05DA1D48BF03F10E0278
:109490006D11D2100DF5A4784FFA85F99345494620
:1094A000404628BF9346FFF7E3FA059B08EB0B0203
:1094B0005B4405998B4240F0E280B7F902304FEAF5
:1094C000CB0B9B4515D9ABEB030B08EB85050022B5
:1094D000CBF12000A845C0F0D7804A46414603980A
:1094E000FFF76CFA012804D04B46039A4046FFF779
:1094F0001FFD5AAD2846029B324652A9FFF760FB7A
:10950000DDE90232294652A8FFF7BDFA2846029B40
:10951000324612A9FFF754FB4FEA840BDDE9023211
:1095200029464AA8FFF7AFFA05EB0B092246514638
:109530002846FFF758FA07F144080AEB0B014846A2
:10954000FFF751FA41462AA8FFF74DFA08EB0B0145
:1095500022A8FFF748FA3B1D29462AAA3046009464
:109560000593FFF7B8FE4B462A4622A92AA8009782
:10957000FFF7C3FE23463A1D31463046FFF728FE6B
:109580003246494628463B46FFF7B3FC0023029982
:1095900052A8CDE90638CDE908A5FFF730FA0299BF
:1095A00080464AA8FFF72BFA8045B8BF80461FFACD
:1095B00088F808F1FF352DB2294652A8FFF73FFA87
:1095C000294610F1000A4AA818BF4FF0010AFFF718
:1095D00036FA002814BF022300234AEA030A0DF1D9
:1095E0001809224659F82A500DF1E809294648463B
:1095F0000DF1C80AFFF7F7F905EB0B015046FFF72D
:10960000F2F921463046FFF733FA01234293A8F1DD
:1096100002080FFA88F8B8F1000F3EDA2346059ADF
:1096200031463046FFF7D4FD3B4632465146484668
:10963000FFF75FFC029A03984946FFF7BFF901283C
:1096400004D0DDE902324846FFF772FC013C64B207
:1096500012AA230663D5049BB3FA83F56D09284645
:109660006BB0BDE8F08F013A13F802C002F800C0F9
:10967000D0E6013D13F8012D08F80520CFE613F8D8
:10968000011D02F8011D14E755F8041D21FA0BF322
:1096900013432B6001FA00F21CE73B463246D7F831
:1096A000A45051464846A847414652A8FFF7C7F97B
:1096B0004146051C4AA818BF0125FFF7C0F900283C
:1096C00014BF022300231D4306AB53F825501DB3DE
:1096D000224629462AA8FFF786F905EB0B0122A8A6
:1096E000FFF781F93B46324622A92AA8FFF701FC81
:1096F000059B00942AAA49461AA8FFF7ECFD534699
:109700004A4622A92AA80097FFF7F7FD3B461AAA66
:1097100031463046FFF7DDFB08F1FF3879E752F8B4
:10972000241059F824304B40049919430491013C0A
:109730008FE770B59DF910401E4623460546FFF79A
:1097400027FC30B9224629463046FFF737F9012871
:1097500007D02346324629462846BDE87040FFF729
:10976000E7BB70BD2DE9F04115468AB00446884636
:109770001C22002103A8FEF7D5FE2E1D95F90070CE
:1097800003232A46414620460293FEF7B7FF33469D
:1097900002AA214620460097FFF79DFD2B46424630
:1097A00021462046FFF795FB0097334605F18402DA
:1097B00021462046FFF7BDFF0AB0BDE8F0812DE944
:1097C000F04793F9006092B004468946104631464E
:1097D00015469846FFF73DF9002840F09180424633
:1097E00049460AA8FEF78AFF43460AAA214602A86C
:1097F000FFF76FFB0AA908464246FEF77FFF434684
:109800002A4649464846FFF764FB08F104074246EA
:1098100029462846FEF772FF3B462A462146204647
:109820000096FFF786FF3B462A46294628460096C3
:10983000FFF77FFF3B462A46214628460096FFF762
:109840004AFD43462A4621462046FFF742FB3B4657
:109850002246214628460096FFF76BFF3B460096BE
:109860002A4621462046FFF764FF2368DB074AD5D6
:1098700033463A4621462046FFF78AFB3146824668
:109880002046FFF78EF806F18043013B54F8230091
:1098900040EACA7044F82300424621462846FEF7B3
:1098A0002DFF3B4602AA294628460096FFF713FDE6
:1098B0003B4602AA294628460096FFF70CFD02A95E
:1098C00008463B462A460096FFF705FD434602AA96
:1098D00021462046FFF7FDFA0AAA3B4610462146DC
:1098E0000096FFF7F8FC324629462046FFF77BF842
:1098F00049462846FFF777F80AA94846FFF773F864
:1099000012B0BDE8F08731462046FFF74AF8C3E7BA
:1099100010B5012203680446984710B1A368013BC3
:10992000A36010BD10B50B689A684B680024C0E9AD
:109930000243C0E9002294782344036192F9034072
:10994000234443614B68036101F10C034361537885
:1099500003F0C003802B04BF0431016110BD4368D4
:109960001A44426011B101399A4201D10120704775
:1099700013F8010B01F8010FF6E72DE9F347002575
:1099800080460F462E462C46D8F8083023B30DF1FA
:1099900007014046FFF7BCFFF0B19DF807C00CF08F
:1099A0007F025FFA82F9A4F12003C4F1200109FAD1
:1099B00003F329FA01F109FA04F20B431CF0800FBA
:1099C00045EA020546EA030604F1070402D1C7E9A5
:1099D000005602E0462CD7D1002002B0BDE8F08747
:1099E000F7B50F4669461646FFF7C7FFB0B1DDE988
:1099F0000013002501F001044A0842EAC37254EA48
:109A000005014FEA530314BFDD431D463B7914BFE4
:109A1000D4431446082B03D1C6E9004503B0F0BD7A
:109A2000042B08D134602246D317AB4206BFA242B2
:109A300001200020F2E7022B03D123B233801AB2B7
:109A4000F2E7012B03D163B233705AB2ECE7002086
:109A5000E4E773B50C4669461646FFF78EFF68B11A
:109A60002379082B0CD1DDE90045C6E90045DDE985
:109A70000023AB4206BFA2420120002002B070BD0D
:109A8000042B04D1009B33601C460025EFE7022B1A
:109A90004FF0000004D1009B33809CB20546E6E7FE
:109AA000012BEBD1009B337003F0FF04F6E737B5D1
:109AB0000D4669461446FFF760FF30B12A79082A3F
:109AC000DDE9003103D1C4E9003103B030BD042A1F
:109AD00018464FEAE37108D123601A460B468B42C1
:109AE00006BF824201200020EFE7022A04D11BB208
:109AF00023801AB2D317F2E7012A03D15BB2237095
:109B00005AB2F7E70020E0E72DE9F3418368074602
:109B1000884623B90026304602B0BDE8F0810DF139
:109B20000701FFF7F5FE06460028F3D09DF8074031
:109B3000220616D504F07F040725BB68002BE9D068
:109B40000DF107013846FFF7E3FE0028E2D09DF84B
:109B5000072002F07F03AB401C43130605F1070505
:109B600002D4C8F80040D6E7232DE6D1D2E773B57A
:109B70000D4601A90446FFF7C7FF064618B900269F
:109B8000304602B070BD94E80F0085E80F000199DF
:109B90008A42F4D3A960A3685B1AA360F0E70000CF
:109BA00030B5044685B01546A9B90268114B9A42F2
:109BB00011D0102D06D82A4669462046FFF7F0FF3F
:109BC00005B030BD102269462046FFF7E9FF0028A6
:109BD000F6D0103DEDE7A368AB4201D20020EFE7DD
:109BE00023682A46204698470028F7D0A3685D1BC3
:109BF000A560E5E75F990700F7B50E4601A907469E
:109C00001546FFF781FFA8B1019A0123D3184FF041
:109C1000000404D2717801F0C001802901D12046EE
:109C200008E031799942FAD329463846FFF7B8FF60
:109C3000019BEC5403B0F0BD73B50D4601A9064677
:109C40001446FFF761FF90B1019AFF2A11D86B7893
:109C500003F0C003802B02F101010AD02B798B4263
:109C600007D32146304601F8012BFFF799FF02B0D8
:109C700070BD0020FBE713B5144669460822FFF7C4
:109C80008FFF18B1DDE90023C4E9002302B010BD45
:109C900013B5144604220DEB0201FFF781FF08B152
:109CA000019B236002B010BD13B5044605291FD8DF
:109CB000DFE801F0030F151E1E1C012201A920463A
:109CC000FFF76EFF18B19DF90430002BF5DB02B0F1
:109CD00010BD082200212046FFF762FFF7E701A927
:109CE000FFF712FF0028F2D0019AF3E70422F1E710
:109CF0000020ECE710B543681A787AB103F10C0242
:109D000042601A7B62B90168C368C0E901128C78AD
:109D10002344036191F903100B444361104620E092
:109D200059781A7901F03004302C1BD15C7B04F097
:109D30003004302C1ED199780269521A0261002237
:109D4000597811F0300F02BF816801318160997B31
:109D5000114402690A44026193F90F301A444261C6
:109D6000012010BD01F0F004202C03D1597911FB22
:109D700002F2E5E701F0C001802908BF0422DFE715
:109D800009B9034B1970034B1B6803B1184770479F
:109D9000C42E0020F82E00201F4B204A1B6800BF55
:109DA00000BF00BF00BF00BF00BF00BF00BF9342A5
:109DB0002FD000BF00BF00BF00BF00BF00BF00BF6B
:109DC00000BF00BF00BF00BF00BF00BF00BF00BF9B
:109DD00000BF00BF00BF00BF00BF00BF00BF00BF8B
:109DE00000BF00BF00BF00BF00BF00BF00BF00BF7B
:109DF00000BF00BF00BF00BF00BF00BF00BF00BF6B
:109E000000BF00BF00BF00BF00BF00BF00BF00BF5A
:109E100000BF0138C3D17047602C00200024F4003B
:109E200018DF70471FB50023CDE90133039368465F
:109E300002230093FFF7F4FF05B05DF804FB000078
:109E4000074A136829B923F00303136043682BB151
:109E5000184723F0010343F00203F6E7704700BF01
:109E600078330020F0B50346186880F308885868F6
:109E7000FF2464B2EFF30585002D01D1A64600470B
:109E80002546064621273FBAF0B4002400250026C7
:109E90000027F0B4F92040B2004700BFF0BD00BF7A
:109EA00013DF7047074A4FF0FF3108B5C2F8801042
:109EB0000346FFF7F5FF20B91846BDE80840FFF755
:109EC000D1BF08BD00E100E0024A1368013B136006
:109ED000704700BF7C33002067DF704763DF704747
:109EE000ADDF7047A9DF7047A8DF7047A6DF704776
:109EF0007FB50023CDF80A30ADF80E3001238DF880
:109F00000A300DF10603ADF80810049302A9044BC2
:109F1000ADF806200593FFF7E9FF07B05DF804FBF5
:109F20008033002010B40D4B024618884FF6FF73A3
:109F300098420FD00A4B1B68DB070BD5094B6024F6
:109F40005A7099701C70084B5DF8044B9989032274
:109F5000FFF7CEBF08205DF8044B7047662C002049
:109F600074330020803300204A33002010B4154B96
:109F7000024618884FF6FF7398421FD0124B1B6899
:109F8000DB071BD5114B60241C7003245C7001247B
:109F90009C70140ADA701C71140C120E9A710A0A61
:109FA000D9711A720A0C090E5A7299725C71084BB7
:109FB0005DF8044B99890B22FFF79ABF08205DF8E2
:109FC000044B7047662C002074330020803300203F
:109FD0004A330020A5DF7047A2DF7047A0DF70473B
:109FE00086DF70477FDF70477DDF70477CDF70471B
:109FF0007ADF704776DF704774DF704773DF704732
:10A0000072DF70476DDF70476CDF704761DF70474C
:10A0100060DF704710DF704748DF70470C4B1B78DC
:10A02000062B10D10B4B1B681A070CD10A4B186872
:10A0300000F0F003302B08D000F0E000A0F1400366
:10A04000584258417047002070470120704700BFB8
:10A05000E00F00F0E40F00F0E80F00F0094B1B7870
:10A06000062B0CD1084B1B681A0708D1074B186840
:10A0700000F0F000A0F13003584258417047002032
:10A08000704700BFE00F00F0E40F00F0E80F00F0B1
:10A09000084B5A6E013A5A6622B907490A7822F0EB
:10A0A00002020A701A6E0132042A08BF00221A66E0
:10A0B000704700BFA43300207033002028DF7047B2
:10A0C00029DF70477BDF704775DF704737B5164B68
:10A0D00018884FF6FF73984210D0144A144D137825
:10A0E000297B0133DBB2994213702C4608D3114906
:10A0F000FFF7EAFF10B1AB6903B1984703B030BD79
:10A10000002313702B7C33B13B21FFF773FF10B199
:10A11000AB6903B198476369002BEFD000228DF83B
:10A12000042001A8E9E700BFFE2E002068340020CB
:10A13000002F00209C33002030B53AB11368DB4378
:10A140000A4D0144884204D1D84330BD4FF0FF335B
:10A15000F6E710F8012B5340082213F0010418BF52
:10A160002C46013A84EA5303F7D1EBE72083B8ED9C
:10A1700010B50A4B1A6A012A0CD8DC6964B19969D6
:10A1800043F2080300221868FFF7D6FF231A58424B
:10A19000584110BD0020FCE70120FAE7AC35002053
:10A1A00010B5084B9A685AB150B9EFF3108172B6E6
:10A1B000054A1C6814605C685460986001B962B616
:10A1C000002010BD7434002000E100E01F4B204A45
:10A1D0001B6800BF00BF00BF00BF00BF00BF00BFC3
:10A1E00000BF93422FD000BF00BF00BF00BF00BF21
:10A1F00000BF00BF00BF00BF00BF00BF00BF00BF67
:10A2000000BF00BF00BF00BF00BF00BF00BF00BF56
:10A2100000BF00BF00BF00BF00BF00BF00BF00BF46
:10A2200000BF00BF00BF00BF00BF00BF00BF00BF36
:10A2300000BF00BF00BF00BF00BF00BF00BF00BF26
:10A2400000BF00BF00BF0138C3D17047602C0020A1
:10A250000024F40010B50A494A788C78531CDBB20C
:10A260009C4208BF00230C789C421FBF03704868C3
:10A2700002EB420200EBC20008BF002010BD00BF8D
:10A280009033002073B5154E736823B3144D6B697A
:10A290000BB300240DF107002C748DF80740FEF776
:10A2A00069F90DF10600FFF7D5FF90B102230370A5
:10A2B0009DF80630456073709DF80700FFF770FF4A
:10A2C00024B9084B4FF48012C3F80021204602B095
:10A2D00070BD0424F0E70824F8E700BF90330020A5
:10A2E0001C2F002000E100E02DE9F347334B344AF6
:10A2F0005B881188334DDFF8E08099420BD8528893
:10A300009A4208D36B69002B56D1002388F800309D
:10A3100002B0BDE8F08798F800403CB16B69002BB3
:10A32000F3D000228DF8042001A841E0264ADFF88E
:10A33000AC901278D5E90163002A18BF1E46D9F8FF
:10A340000430002B36D0042E2DD9204F7B698BB3DF
:10A350007B7C8DF80440012B01A80CBFB2464FF066
:10A36000000AFEF707F90DF10300FFF773FFC0B114
:10A3700001230370164B4760D3F80435C0E904A4E9
:10A38000C0E902369DF8033089F801309DF80400D9
:10A39000FFF706FF44B90F4B4FF48012C3F80021BA
:10A3A000B3E70424F2E70724AB69002BADD02046C5
:10A3B0009847AAE70824F7E70122B3E73C2F0020DB
:10A3C0009C330020002F0020683400201C2F002028
:10A3D0000010014000E100E0FC2E0020903300203E
:10A3E0000D4B0E494FF4003210B5C3F88020012404
:10A3F0004FF48033C1F848332F20C1F808334C6044
:10A40000FFF7E4FE064B8C602F2000211960FFF758
:10A41000DDFE044B197010BD00E100E000100140AA
:10A42000643400204E340020F8B5124C124D2646FC
:10A4300022782B789A4200D1F8BD23780F48104A31
:10A44000078812680F48DBB219B202EBC10C006832
:10A4500052F83120BCF8041003FB070090470A4A69
:10A4600023781288DBB29A4286BF0133DBB2002325
:10A470003370DDE71C3400200C3400201834002039
:10A4800014340020103400201A34002038B5064C53
:10A49000064D636E042B00D038BD2846FFF77CFCC8
:10A4A000FFF7C2FFF5E700BFA4330020A08601003C
:10A4B0005B689A68054B9A4206D1D0E901230449AA
:10A4C0000132013B0A604B60704700BF5CCD070062
:10A4D000E82E0020BFF34F8F0549064BCA6802F4EF
:10A4E000E0621343CB60BFF34F8F00BFFDE700BFB7
:10A4F00000ED00E00400FA0508B5FFF7EBFF0000EF
:10A500002DE9F743244E254F33683A68B3FA83F5B3
:10A510006D09002A3BD0DFF8888098F8003003F0FE
:10A52000FF046BBB01A8FFF777FD052823D008B116
:10A53000FFF7D0FF3B6801989847F5B9184DDFF851
:10A540006480DFF864902B78D3B9B8F80030ADF8A8
:10A550000230D9F800300DF102011846FFF756FD20
:10A56000052810D00028E3D1326818469047002C07
:10A57000E9D12546CFE70124DFE70125002CCCD027
:10A5800003B0BDE8F083002CFAD10124F1E7002BE1
:10A59000F6D00124D2E700BFF42E0020543400206E
:10A5A00050340020F02E00206C34002008B509B192
:10A5B000FFF790FF034B1B781BB1BDE80840FFF786
:10A5C0009FBF08BD4F34002008B5FFF783FF08295F
:10A5D00010B501D0FFF77EFFD0E90030BDE8104094
:10A5E0001847000008B5084E084CA41BE4080025D5
:10A5F0000436AC4203D056F83530984708B1FFF71F
:10A6000069FF0135F5E700BF802C0020882C002071
:10A610004FF0A043D3F810056FEAD02000F00100FE
:10A620007047000070B50C4C00EB400023184FF051
:10A63000A0425D78205C05F5E073032642F82360B4
:10A64000C0F300100123AB4088420CBFC2F80C35A8
:10A65000C2F8083570BD00BF44CF070010B50446EE
:10A660002620FFF7DFFF21462520BDE81040FFF739
:10A67000D9BF000070B543F208031C68164B196877
:10A68000A1F54051091B814224D3144B144E1D6A7D
:10A690003460012D1AD19A6902F6FF7222F47F62AA
:10A6A00022F00F02891A88424FF0000103D9C3E952
:10A6B0000451183304E02244C3E904153260243302
:10A6C0000022C3E901221860104670BD0022C3E9D0
:10A6D0000422EEE70420F8E714100010AC35002047
:10A6E0006C33002070B59CB000230022109300232F
:10A6F000CDE912234C4B4D4A4D4C4E4DCDE9142320
:10A700004D4BCDE916434D4BCDE918534C4B1A93A5
:10A7100003F17453A3F52303A3F692431B9309B1EA
:10A72000002852D0044645180026A54250D1454D78
:10A730002C68002C49D0109A1CA9531C372A0A44B3
:10A740004FF0800102F8701C4FF0000260D8382BE7
:10A7500057D1DDE9122310980821E1FB00231046B0
:10A76000194612BACDE912010F9269461A0A8DF8FC
:10A770003B308DF83A2008461A0C1B0E8DF8392014
:10A780008DF83830FDF71CFF621E00231B99D9405D
:10A7900002F8011F1A99D94011711999D940117203
:10A7A0001899D94011731799D94011741699D94045
:10A7B00011751599D94011761499D9400833202B79
:10A7C0001177E3D16B60002000E00E201CB070BD5B
:10A7D000109B14F8011B1CAA1A440133402B02F8E9
:10A7E000701C1093A1D169466846FDF7E9FE129BE3
:10A7F000139A109613F5007342F10002CDE912325C
:10A8000093E70DF803200133A1E70DF8032001338E
:10A810003F2BFAD969466846FDF7D2FE382200215F
:10A820006846FDF77FFE94E785AE67BB67E6096A79
:10A8300072F36E3C7F520E513AF54FA58C68059B22
:10A84000ABD9831FE82E0020044A00230360436035
:10A850008360C2E90C33C2E904337047AC35002091
:10A8600010B50C494A6E042A044611D00B6E1344ED
:10A87000032B02F101024A6688BF043B182202FB47
:10A88000031318460021FDF74DFE2060012010BD86
:10A890000020FCE7A433002030B5044685B00D4607
:10A8A000102200216846FDF73DFE237A012B0AD0D5
:10A8B000022B0ED063680193236829469B68684683
:10A8C000984705B030BD23690293A38AADF80C30D8
:10A8D000F0E70123A2898DF80030E389ADF80A2062
:10A8E000D31AADF80830E5E738B51C4B5A6E194657
:10A8F0005AB31C6E182202FB04331A7A012A07D0BD
:10A90000022A23D018460921BDE83840FFF7C4BF0A
:10A910001825D88A9A8A05FB0414D4E90314121A5C
:10A92000B2F5806F4FEA80000144B4BF92B24FF499
:10A9300080622044FFF7C4FB11280BD1084A13782A
:10A9400023F0020343F00403137038BD9889FFF726
:10A95000B5FBF1E70028F8D0D4E700BFA43300200E
:10A960007033002038B52A4A13780146980742D53B
:10A97000284A146E1820022900FB042005D0032960
:10A980002DD0BDE83840FFF7AFBF234B0021197031
:10A99000037A012B0CD0022BF3D18389028A013375
:10A9A0008381C38901339BB29A42C381E9D111E00B
:10A9B000858AC38AE91AB1F5806FB4BF89B24FF4B2
:10A9C00080610B4418219BB201FB04229D42D3827B
:10A9D000D7D10021FFF760FFFFF75AFBD1E70E4AFE
:10A9E00013780133DBB2032B01D81370C9E70023BE
:10A9F00013700821EEE75907C3D50649496E03F0E5
:10AA0000FB0313700029BCD043F00203EDE700BF45
:10AA100070330020A43300204C340020054A137802
:10AA200013F0060F04D143F002031370FFF75CBF6D
:10AA3000704700BF703300202DE9F043494ED6F82F
:10AA4000009019F0040F85B0054614464DD019F05A
:10AA5000020F40F0818049F001033360424B1B78C4
:10AA6000DB073CD5414F424B9F423AD3414B9F427B
:10AA700037D2002837D0C0F30B0373BB3B68984232
:10AA800004D2052029F0010333601FE08AB27B68FD
:10AA900000EB02329342F4D31FFA81F8B8F1000FB1
:10AAA00019D06846FFF7DCFE98B1009BC3E900743B
:10AAB000009B02222D0B1A729D81A3F81080FFF7D4
:10AAC000ADFF336843F001033360002005B0BDE8FB
:10AAD000F0830720D6E70420D4E70620D2E7012040
:10AAE000D0E70220CEE70320CCE7C0F30B03ABBBDB
:10AAF000214E0F464FF0020C3246C6F804C5D2F87C
:10AB000000E4BEF1000FFAD0C2F80805D2F800E464
:10AB1000BEF1000FFAD0C2F80435D6F800E4BEF159
:10AB2000000FFAD0013F00F58050E6D105EB013669
:10AB3000B4B1394610226846FDF7F4FC310B01230D
:10AB40002D0BADF80A10684639468DF80030019497
:10AB5000ADF80850A047B8E70A20B7E70620B5E7E8
:10AB60002046B3E77833002070330020702C00209B
:10AB7000702C0020802C002000E001402DE9F043E3
:10AB80000F4646491C460B6813F0040F85B0054676
:10AB9000884646D09E0777D443F001030B60404BB4
:10ABA0001B78D80772D53F4E3F4B9E4270D33F4B28
:10ABB0009E426DD21FB9032005B0BDE8F083002D81
:10ABC000F9D047EA0503990701D00620F4E7336876
:10ABD0009D425FD393B2716805EB8303994259D3C9
:10ABE0001FFA82F9B9F1000F01D10420E4E76846A9
:10ABF000FFF736FE98B1009BC3E90064009B012279
:10AC00001A72C3E90375A3F81490FFF707FFD8F889
:10AC1000003043F00103C8F800300020CCE70720E3
:10AC2000CAE7002FC7D00028C5D047EA00039B071A
:10AC3000CBD1002AD9D01E4B0121C3F80415D3F87B
:10AC400000140029FBD01A490023084657F8236056
:10AC500045F82360D1F80064002EFBD001339A42FE
:10AC6000F4D10023C1F80435D0F80034002BFBD018
:10AC700000268CB1314668468DF80060CDE901456B
:10AC8000ADF80C20A047C8E70A2095E7012093E71C
:10AC9000022091E705208FE720468DE778330020DA
:10ACA00070330020702C0020702C0020802C00209D
:10ACB00000E00140F8B51E4C1E4F0646254623789D
:10ACC0009BB9012323701C4B1C4C1E60FFF7DEFB5D
:10ACD000002201212046FFF7AFFE07280246F5D0EB
:10ACE00048B100232B700320F8BD3846FFF754F815
:10ACF000FFF79AFBE3E7124C124F134E5821201D29
:10AD0000FFF71AFA214620604FF4AE720E480B4C42
:10AD100001F068FFFFF7BAFB3B4657223146204659
:10AD2000FFF72CFF0728F5D00028DDD0D9E700BFBA
:10AD3000C42E0020A0860100F82E002000F007009D
:10AD4000AC350020819D0700583700202DE9F04FD9
:10AD50001E4E1F49726B336B02F6FF74E41A0C40EF
:10AD6000A50805F6FF7585B003F580570D4003EB88
:10AD700000080AB1934226D04FEA95094FF0010A24
:10AD80004FF0030B6846CDE900A8CDE90279FFF743
:10AD900047F8A8B96846CDE900B7CDE90289FFF7C1
:10ADA0003FF868B9A542736B8CBF0446641B1B1B3C
:10ADB00000202F44A8443363FFF77CFF002CE1D12F
:10ADC00005B0BDE8F08F0020FAE700BFAC350020E9
:10ADD00000F0FFFF7FB5124B0C685B6B1D18E41A87
:10ADE000032300930F4BA4086846CDE90135039473
:10ADF000FFF716F8064638B90846FFF725FD304636
:10AE0000FFF758FF04B070BD102200216846FDF71F
:10AE100089FB6846CDE90154FFF702F8F2E700BF6D
:10AE2000AC3500200080070030B54268527802F04F
:10AE30000F01082987B003460FD103691C6800255C
:10AE40000CB907B030BD214625736846FEF76AFD90
:10AE50006846FFF7E9FFA468F2E712F0C00120D1CD
:10AE600002F0300010280ED15A6911705A68186922
:10AE70005378946803F00F03072B09D1014620464D
:10AE800000F017F8DDE79006F0D55B691970D8E798
:10AE90001279214614B101F0A5FED2E7FDF742FB7D
:10AEA000CFE78029CDD10069002192060160C8D585
:10AEB000EBE77FB50023CDE902318378194490F99F
:10AEC00003300491194403780591CDE900003BB1AA
:10AED0006846FFF7A9FF6846FEF70CFF0028F7D188
:10AEE00007B05DF804FB00002DE9F04355686B786E
:10AEF00013F0C00489B006468C46174603D0402C98
:10AF00006AD000240AE003F00F025E4903F0300328
:10AF1000102B51F8228020D004D8CBB1204609B0A4
:10AF2000BDE8F083202B1ED0302BF7D17B69297828
:10AF30001970072A0AD17B6838691A792146FDF70A
:10AF4000F1FA7B6839699868FFF7B3FF3A6940E026
:10AF50003A692946C0470446E0E77B6901221A7036
:10AF60003A697968F6E7BCF1020FD7F8149024D15A
:10AF7000042A22D804A9FEF7FAFD04460028C0D00E
:10AF8000069B2BB1796899F800304A799A4205D826
:10AF9000059B7360069B002BC0D0B2E708793A6925
:10AFA00000FB032204A8C04728B199F80030013300
:10AFB00089F80030E4E70446EAE799F800306A7956
:10AFC0009A429ED93A692979581C89F8000001FBF8
:10AFD000032279683046BDE7D2F81080454655F81F
:10AFE000043B13B9FEF760FEB5E7022914D104A9AA
:10AFF000FEF7BDFD002884D0D8F8003079682A46D5
:10B0000004A89847044600283FF47BAF069B002B1A
:10B01000F2D1059B736081E701292BD04CB24CB172
:10B0200005297FF46EAF04220DEB0201FEF7B8FD97
:10B03000042424E00DF1040901340B2C3FF461AF2A
:10B04000012249463046FEF7ABFD00283FF459AFD8
:10B0500019F9013B002BEFDB0B4B049301ABCDE95E
:10B06000053400230793D8F8003079682A4604A8ED
:10B07000984770E7082201A9FEF792FD08240028EE
:10B08000EAD13EE72CCC07005F9907002DE9F04F8D
:10B090008B788FB00025CDE904521A4491F9033022
:10B0A0000692CDE90055CDE902111A4404460792F3
:10B0B0004FF00108A3682BBBDDE9033402A85D78DB
:10B0C000FEF718FE0028F7D115F0300F03D1039BCF
:10B0D0001B7803B10134002C65D063090022934230
:10B0E0005BD10EAA02EB830304F01F044FF0FF3084
:10B0F000C4F1200420FA04F453F8380C231A5842FF
:10B10000584108E008A92046FEF7FEFC30B9A368C4
:10B11000002BD1D000200FB0BDE8F08F089EDDF8E5
:10B120000CA0002EC8D0F70806F00706039B1A787B
:10B13000974204D15B7803F00F02082A58D102A885
:10B14000FEF7D8FDDDF80C90CA45EFD1BD420DD811
:10B15000039A537803F00F03082B29D002A8FEF7B7
:10B16000C9FD039B9945F3D14FF0FF353146204689
:10B17000FEF79AFD00289DD1CCE79B681B789F4283
:10B1800033D1494608A8FEF7CDFB89F80C8008AA00
:10B1900031462046FFF7A8FE25E05DF82210013178
:10B1A000B8D101329BE70120B5E79A45DED081E7AF
:10B1B0001578BD42DAD8069BD4F808A0D3F80090E1
:10B1C000A368B9F1000FF0D09A457FF473AFD9F8B6
:10B1D0000030D3F800B0BBF1000FCED033463A4672
:10B1E00049462046D847002894D0D9F80890E7E788
:10B1F00013F0300F0FD1049B3F2B0CD85A090EA926
:10B2000001EB820203F01F0352F8381C08FA03F323
:10B210000B4342F8383CD4F80C90B9F1000F04D03D
:10B2200002AB324639462046C84702AA314620467C
:10B23000FFF75AFE9EE7F0B585B00E468C6869466A
:10B2400007461546FEF793FC88B1B06878B173786D
:10B2500003F03003202B03D129462046FFF729FEB7
:10B260002A4621466846FFF711FF019B7B6005B027
:10B27000F0BD000070B50D4B0D4C9A6B0D4E0E4D90
:10B280000E4921605C33C4E901320D4BE3600D4B84
:10B29000002231462846C3E90022FFF70AFE324663
:10B2A00029462046FFF7F2FE70BD00BFAC350020F6
:10B2B0004837002080340020D8CD07005F99070070
:10B2C000B1A40700E82E00202DE9F3410024064632
:10B2D0000DF107000D4617468DF80740FDF74AF9B6
:10B2E000204B214A18781178CBB2204909888B422B
:10B2F00038BF0133C0B238BFDCB2A04228D01478C6
:10B300001378DBB2994286BF0133DBB2002313709E
:10B310009DF80700FEF744FF4FF6FF739C421ED0D6
:10B32000134B1B6803EBC40843F834709EB195B10E
:10B33000104B1888104B1B682A46314604FB00301E
:10B3400001F050FCA8F80450002002B0BDE8F081E4
:10B350004FF6FF74DCE70020A8F80400F5E70420AE
:10B36000F3E700BF1C3400200C3400201A34002006
:10B3700014340020183400201034002007B5084B86
:10B380001B88072BCDE9000107D9064A082168462A
:10B39000FFF79AFF03B05DF804FB0920FAE700BF4E
:10B3A00018340020CFA507000021024A0846FFF705
:10B3B0008BBF00BFADA5070010B5114C21684A072F
:10B3C0001BD441F004030F482360FEF7E5FC0E4B4D
:10B3D00018884FF6FF73984204D01321FEF70AFE37
:10B3E00048B110BD8B0706D5FEF706FE0028F8D140
:10B3F00041F006012160FEF745FF0020F1E700BFA4
:10B4000074330020C0D40100662C002070B52A4E91
:10B41000356815F002018AB04CD1102201A8FDF761
:10B4200081F80B23ADF80230244B059345F6021347
:10B43000ADF818300DF10201FE230DF11D008DF85D
:10B440001A30FEF7D1FD044648BBBDF802100B29A7
:10B4500028D84B1C8DF81B30092319448DF81C305B
:10B4600089B200231A46C9B205A8FEF7C9FD0446F1
:10B47000A8B98DF8040002908DF80C002823ADF8CF
:10B48000100001A8ADF80E30FEF7B8FD044630B943
:10B49000014645F002050120FFF7E0F8356020463F
:10B4A0000AB070BD0C238DF81B3008238DF81C30BA
:10B4B0001421D6E70024F2E77433002002010603CA
:10B4C0002DE9F04194B04FF404330493FEF7AAFC45
:10B4D0000446002840F03D81A748FEF7E1FC044601
:10B4E000002840F03681A54BA54A1A60A54B502292
:10B4F0001A80A54BA54A1A60A54A1368C3F34033C6
:10B500001BB14FF40051C2F88010A24904A8FEF705
:10B5100081FD9F4A28B113B14FF400531360FEF729
:10B52000D9FF9D4B0121197092F816335806F6D5B4
:10B530009A4B9968002900F010811A6842F4800241
:10B540001A60162200210DF13600FCF7EBFF0022F5
:10B55000139240F20112ADF83C201722ADF84420BE
:10B560008F4A01920123019A089208A90DA8ADF80B
:10B5700034308DF83E30FEF74BFD019A044600282A
:10B5800040F0E780874A88491160CDE90D0011221B
:10B5900008A88DF81020FEF735FD0446002840F07D
:10B5A000D8809DF8212008A801328DF82120FEF7CF
:10B5B0002BFD0446002840F0CC8007227B4904A8DC
:10B5C000FEF714FD0446002840F0C38078494FF090
:10B5D000C8720DA8CDE90D12FEF70AFD0446002839
:10B5E00040F0B780734A8DF80A304FF6FF71118032
:10B5F0004FF65962ADF8082002A96F4A1846FEF7C7
:10B60000EDFC0446002840F0A4806C4B04AC03F130
:10B61000100518685968224603C20833AB42144625
:10B62000F7D1654D04A8A91CFEF758FC0446002874
:10B6300040F08F8001461C220DA8FCF773FF9DF897
:10B640003430ADF8004043F004038DF83430AB786B
:10B650008DF80E300223ADF80C301423CDE90A44E6
:10B66000ADF82C302B460C94274604F0F80444F037
:10B6700003044FF0110803AE08AA0DA933F8040B18
:10B680008DF802408DF801800896CDF824D0FEF7A1
:10B69000A3FC044600285CD101461C220DA8FCF73F
:10B6A00041FF9DF83430ADF8004023F0180343F01B
:10B6B00018038DF83430AB788DF80E300123ADF8D7
:10B6C0000C3007F0E80343F013038DF80230172322
:10B6D000CDE90A44ADF82C302B4608AA0DA933F861
:10B6E0000C0B0C948DF801800896CDF824D0FEF751
:10B6F00073FC044668BB324A324D136843F00103C1
:10B700001360014618220DA8FCF70CFF40F6CD424D
:10B710004FF48043CDE90E2303238DF840302A4BAC
:10B7200013930DAC0FCC0FC594E80700274B85E8A9
:10B73000070027481F70FEF7C5FC044648B9254B93
:10B740004FF6FF721A80244B1F70244B5B6843B97D
:10B750000824204614B0BDE8F0814FF48003136044
:10B76000EFE61F4B1A7C002AF2D11E4A5F745A6121
:10B77000FFF74CFE0446ECE7008007006C34002025
:10B780006C2E0020F02E002064330020A9B30700A7
:10B7900000E100E0C9A507004F3400207434002008
:10B7A000002C0020F42E0020E9B7070050CC070041
:10B7B0000C001800662C00204A3300201CCC070027
:10B7C00074330020002F0020F9A40700FC2E002075
:10B7D0009C330020FE2E002068340020903300208F
:10B7E0001C2F0020CDA007002DE9F04F0388112B5E
:10B7F0008DB0044639D010D8102B23D02388142BB9
:10B8000000F0938357D8102B00F0B08045D8022B5E
:10B8100000F0C3800DB0BDE8F08F122B36D0502B56
:10B82000ECD1A74DC288EB899A42E7D1038A022B5B
:10B83000E4D1837CD90715D4FEF724FD0028DDD0A0
:10B84000AB691FE09F4B82881A8000F1100303CB85
:10B850009D4A9E4B1060516000221A70984BDB8904
:10B86000002BCBD1FEF740FDC8E7964B4FF6FF7299
:10B870001A80964B00221A70FEF704FD0028BDD0F6
:10B880008F4B9B69002BB9D09847B7E700F10803AD
:10B8900003CB8D4A10605160E4E7112B73D0132B5A
:10B8A000B8D18B4800231A4685210088FEF79AFB01
:10B8B0000028AFD06AE0522B00F03E8346D8502BD0
:10B8C00000F04183512BA5D1A579002DA2D01022E3
:10B8D000002108A8FCF726FE022D9BD17D4E22896F
:10B8E000B3899A4296D1A37B043B022B92D99DF84F
:10B8F0002630318A43F001038DF82630238AADF8D3
:10B900002830638AADF82A3004F114030B93002326
:10B91000ADF81A3005AB07936D4B1D8802228DF8E8
:10B920002020ADF81820284606AAFEF753FB002871
:10B9300039D19DF81430DA0735D440F2FD1308A947
:10B940002846ADF82430FEF7CFFA63E7552B00F018
:10B950001C84562B7FF45EAFA379002B7FF45AAF83
:10B960005B4B13211888FEF745FBA1E7012100205E
:10B97000FEF774FE564BA2881A80574A136823F0CC
:10B980000203136046E7FFF741FD08B1FEF7A2FD91
:10B990004F4B4FF6FF721A803CE74D4B0021188841
:10B9A000FEF79AFA84E7002308A92846ADF8243068
:10B9B000FEF79AFA00287FF42DAFCDE908000A902F
:10B9C000207D431E052B00F2AE82DFE813F0060057
:10B9D000350245029F00AC025B02638A062B01D050
:10B9E000032116E03D4BD4F816501A883C4B0A95BB
:10B9F0001A80637D0993012293428DF820200CD197
:10BA0000384A1370374B1C78012C0AD0022C1BD0FB
:10BA100005210120FEF786FAFCE6022BF0D0072173
:10BA2000F7E7002DDCD0B5F5807F46D82E4E2F4BA2
:10BA300000271C22394606F13C001F70FCF772FDFE
:10BA40003763B5630121E4E7002DC9D0C5F30B03CB
:10BA500033B1254B264A5B6D12682B449342BFD10C
:10BA6000B5F5805F29D8214B1B78002B4CD01E4B9D
:10BA70001F4A586D12682918914245D8DA6C18652A
:10BA8000C3E911521B4A186313781B4C013303F0AE
:10BA900003031370194B00221A802368184A0133DC
:10BAA0002360184B1B6801211844FEF7C5FF0028CE
:10BAB000C8D02368013B2360AAE70421A9E700BF9F
:10BAC000002F0020FE2E00203C2F00206834002094
:10BAD000662C00204A330020743300209833002065
:10BAE0009A330020642C0020AC35002069340020FB
:10BAF00068330020442F00207C330020483300208E
:10BB0000C99E07006C330020082182E703238DF8CB
:10BB10002030974B1C78012C04D0022C00F0D680EA
:10BB20000524ADE0934FD7E90E21914240F0828188
:10BB3000914E3378002B40F0A380FFF79BFB012848
:10BB4000EED18E4B93F874201C46002A00F0B98089
:10BB500093F87A30002BE3D0894DD5E90001A8B1E4
:10BB6000A1B194F8DB3013B194F8DC3073B994F8D8
:10BB700084305BB1D4F88830342B07D194F88CC072
:10BB8000804A002343F20C0E634501DB0A2477E070
:10BB900052F8049BBEF80080C14500F0FC820133DE
:10BBA000F2E794F87C30002BF0D0BA68D4F88030FB
:10BBB0009A42EBD894F8E830002BE7D1724B2B6017
:10BBC00020236B60FEF78EFD0028DFD194F8E9702A
:10BBD0006E4B6F493A46184601F004F86D4A402F03
:10BBE0000346C2E900079BD12968002998D011F0CB
:10BBF000030795D1684A00926A686848FDF7E2FB3E
:10BC000000288DD0664D94F8A1302F60032BBDD84D
:10BC1000DFE803F00C39294194F87C30002BB5D0D3
:10BC2000FA68D4F880309A42C4D3AFE794F8B030C1
:10BC3000002BABD0D4F8B4302B605A4B524C03F1EC
:10BC4000200718685968224603C20833BB421446CD
:10BC5000F7D1286880B3FEF70DFD80B90124FFF706
:10BC600029F834700CE094F8A830002B8ED0D4F86A
:10BC7000AC202A604C4BC3F5FC239A42DDD9042446
:10BC800021460420C6E694F8A230002B3FF47EAF94
:10BC9000D4F8A430D0E794F8A830002B3FF476AF66
:10BCA00094F8A230002B3FF471AFD4F8A430D4F84C
:10BCB000AC20991829600BB90324E1E7002AD9D1F7
:10BCC000FAE71B78002B7FF461AF29E7294CD4E910
:10BCD0001423616CD31A9942264640F0AB80A36CC2
:10BCE00062650020E3646064FEF7E4FF2C4B216D85
:10BCF0001A689142984632D12C4C2368002B30D1DF
:10BD00001E4D95F8B930032B2ED11D4F1E4B3B60B5
:10BD1000274BD8F8001018684FF02009C7F8049096
:10BD2000FEF7E0FC4A46002805F1BB01386814BF65
:10BD30000A24012400F048FF002818BF0524736975
:10BD4000A3B1012B7FF422AF1A4B012C6ED195F8D1
:10BD5000A120032A68D8DFE802F031555B61012495
:10BD60008EE7FEF761FBC8E70A24E8E7124BECE731
:10BD7000642C0020AC350020693400208034002081
:10BD8000E82E002010350020C82E002008370020A3
:10BD90006A350020BC2E002058CC0700D4CF070005
:10BDA000683300203B350020008007007C330020F2
:10BDB0006C330020D0350020C435002001229A6069
:10BDC000D5F88020B260B26C5A60D8F800201A60B2
:10BDD00000212022B248B34DFCF7A4FBB222FF2180
:10BDE000B148FCF79FFB00233363B04E2846FEF7B3
:10BDF00061FF11287FF444AF3046FDF7CDFFFEF719
:10BE000013FBF3E7A5229A60D5F8A4207263DAE762
:10BE1000AA229A60D5F88020F260D4E7AC229A601A
:10BE2000D5F8A4207263F5E70A24CCE70022C3E921
:10BE30000122CCE7082423E7638A032B02D00321E5
:10BE40000220E7E5A27D637D43EA0223984A13803E
:10BE5000984A01211380F3E704238DF82030964B94
:10BE60001B78012B04D0022B08D005210320D1E53B
:10BE7000924BD3E90F01FEF779F8CBE48F4B186DA5
:10BE8000996CF8E7638A022B02D003210620C1E5F2
:10BE9000637D09930622012B8DF8202009D1864A63
:10BEA0001370854B1B78012B07D0022B35D0052151
:10BEB000ECE7022BF3D00721E8E7804BD3E90F1220
:10BEC0004FF480704FF6FF739D423FF4A3AC7C4B60
:10BED0001B68DB077FF59EAC7A4B000A6024187163
:10BEE000080A1C70D97106241872080C090E5C70BF
:10BEF00099720124110A9C70DA7200241973110CD2
:10BF0000120E587259739A73DC705C719C710F2217
:10BF1000B1892846FDF7ECFF7CE4684B4FF4805074
:10BF20009A6C196DCEE7032174E500231A46194671
:10BF3000A088FEF755F8BBE400231A461946A088EE
:10BF4000FDF7D0FFB4E4604BE2889B889A427FF40F
:10BF500061AC0223002508958DF82030564B268AC7
:10BF60001B780A9604F11207012B099715D0022BB2
:10BF700032D0AA464E4B1E88002E3FF44BAC4D4C9F
:10BF80002388013B9BB22380002B7FF443AC2946DE
:10BF90005046FDF7EBFF26803CE4484CD4F83CA02B
:10BFA000A36B06EB0A029A4201D9256CE2E70AF17B
:10BFB0005C0032463946204400F014FEE06B04F188
:10BFC000400206EB000A31463846C4F83CA0FEF7B2
:10BFD000B3F805462064CDE73C4B384C1B78D4F8C9
:10BFE00050A0A56C002BC5D0B6F5807FC2D8636D7C
:10BFF000626C06EB0A09A9EB03039342BAD804F179
:10C00000480231463846FEF797F83149DFF8C8A0B4
:10C010000B78BAF80020A0644FEA032B2D4BC4F82C
:10C02000509005460BEB02001844B318FF2B039306
:10C03000884659D83246394600F0D4FD039BAAF809
:10C040000030CA46244E3288002A93D0636D206B9C
:10C05000616CD31A03448B428CD3204B204FD3F80E
:10C0600000C03B6898F800E01A49013303323B6096
:10C0700092081C4B01EB0E216044FEF77FFD002867
:10C0800079D1236B32881344236398F8003001334D
:10C0900003F0030388F80030002333806AE700BF11
:10C0A000E4350020E5A5070008360020A086010041
:10C0B000983300209A330020642C0020AC350020F7
:10C0C00074330020803300204A330020693400207C
:10C0D000442F0020482F0020483300206C330020DC
:10C0E0007C330020C99E0700C2F580739BB21A46BC
:10C0F0003946039300F076FD039B206B2E49F61A18
:10C100001F440A962D4B2E4E09971F6833684FF433
:10C1100080720133AAF8002033604022294B594431
:10C120003844FEF72BFDE0B9BAF80020236B134426
:10C130002363CA4698F80030234F0A9E013303F068
:10C140000303002288F800303A80002E3FF47AAFD3
:10C1500019480999324600EB032000F043FD3E8068
:10C1600070E73368E56CD4F854A0A564013B3360F4
:10C17000C4F850A0DEE73B68E56CD4F854A0A56491
:10C18000013B3B60C4F850A07FE71721A088FDF772
:10C19000A7FEFFF78DBB94F8A120032A3FF6F6AC6B
:10C1A00001A353F822F000BFA3BB0700B5BB0700F3
:10C1B00019BC070019BC0700482F00206C33002071
:10C1C0007C330020C99E07004833002008B5074B88
:10C1D0001B681BB1984740B1FEF77CF9044B1B78F4
:10C1E0001BB1BDE80840FEF78BB908BD64330020E1
:10C1F0004F34002008B5FDF731FF10B14F4B504AC6
:10C200001A60FDF70BFF28B14E4B4F4A1B68C3F372
:10C2100042331360FDF722FF20B14C4AD36823F06C
:10C220008073D360FDF7FAFE40B14FF080430022E7
:10C23000C3F80C21C3F81021C3F83825FDF70EFF11
:10C2400010B1434B03221A60FDF708FF40B1414B88
:10C2500005221A6001229A6700229A603F225A60E2
:10C260003D4B1B78062B50D13C4B1B681B074CD118
:10C270003B4B1B6803F0F003502B46D14FF080522C
:10C28000384BD2F80414C3F82015D2F80814C3F8B8
:10C290002415D2F80C14C3F82815D2F81014C3F8DA
:10C2A0002C15D2F81414C3F83015D2F81814C3F8AA
:10C2B0003415D2F81C14C3F84015D2F82014C3F872
:10C2C0004415D2F82414C3F84815D2F82814C3F83A
:10C2D0004C15D2F82C14C3F85015D2F83014C3F80A
:10C2E0005415D2F83414C3F86015D2F83814C3F8D2
:10C2F0006415D2F83C14C3F86815D2F84014C3F89A
:10C300006C15D2F84424C3F87025FDF787FE28B1D8
:10C31000154B164A1B6803F04F031360144AD2F8FA
:10C32000883043F47003C2F88830BFF34F8FBFF3F7
:10C330006F8F104B104A1A6008BD00BF74C00740D1
:10C340000DF0ADBA440200103C050040F0ED00E0F5
:10C35000A005004010560040E00F00F0E40F00F090
:10C36000E80F00F000C0004058020010E40E00404A
:10C3700000ED00E0602C00200090D00373B5002396
:10C380000DF102008DF80230FCF7F4F8264B1B7813
:10C3900003F0FF04002B41D1244B1A68002A3DD042
:10C3A000234AD2F80813C90738D51C601B68214DF1
:10C3B00001930DF10300019BD2F808658DF803404D
:10C3C000FCF7D8F86A6829681F2A98BF541CA14254
:10C3D000F6B26C6004D1202C14BF611C00212960CE
:10C3E00015499DF803008E542A6894423ABFC2F161
:10C3F00021021319A31AAA689A4238BFAB60FDF74D
:10C40000CFFE6B682A681F2B94BF013300239A422A
:10C4100001BF074A0123C2F8083353609DF80200A8
:10C42000FDF7BEFE02B070BD4F34002000D10040C9
:10C4300000D00040403400201D3400202DE9F04F92
:10C44000AF49B04AB0480B68007887B004931378BE
:10C45000984200F0B0800133DBB2022B08BF00230A
:10C4600013701278A94B53F82240049B234423F005
:10C470007F430B6001230193A54AA6481378D0F8A7
:10C4800000C050780390506892780592A24A0290BA
:10C490000020D1F8009092F8008019466246864646
:10C4A0008246039DA94240F08980BEF1000F05D06D
:10C4B000994981F800809249C1F80090954900B1EE
:10C4C0000A6001980A68002840F0C980BCEB0202AB
:10C4D00018BF0122019200268F4AD1F800A01278DD
:10C4E0000492874A4FF0000CD2F800905046614603
:10C4F0004FF0010BE646002E40F0B680039A9A42B8
:10C5000040F0D18009B1824B1A70824BBCF1000F10
:10C5100000D018601B689A4502D1019A002A44D0C5
:10C52000002B00F01A81D3F800907C4C744BD4F8A7
:10C53000046519687A4F751A3B7825F07F450335F5
:10C54000A3B94FF48033C4F84433C4F80433754BB3
:10C550004FF400324FF00108C3F880212F201A60F9
:10C56000C4F80080FDF732FE87F80080A9452CBF93
:10C570004944491921F07F41C4F84015D4F80435E5
:10C580009B1B23F07F43891B033321F07F418B42A8
:10C590000BD9D4F80435C4F840352F20FDF716FE2A
:10C5A000604B4FF40032C3F800215B4B00221A703D
:10C5B00007B0BDE8F08F002401945DE7029E01EB17
:10C5C000410506EBC5070131059EC9B2B14208BF5E
:10C5D0000021029E16F83550022D0AD0032D7FF45B
:10C5E00060AF002A3FF45DAF82F810A00120D2694D
:10C5F000F7E7D7F804B015461646002D3FF451AFC3
:10C60000AB4500F0AD802E46ED69F6E70120B4E0C1
:10C61000D2F800C0A44505D905B10A60ACEB04040A
:10C62000146059E7A4EB0C046044D2F80CC0C2F8C3
:10C6300000E0D2F81C80BCF1000F07D0049DD66149
:10C64000054425F07F45C2E9015C164601254246B6
:10C65000002ADDD1002D3FF43FAF0A603CE7002502
:10C660002E462846AE46F3E73246F669D2F80480F5
:10C670002D4C9768A8EB090525F07F45A54234D8D5
:10C680003D441560C2E901EE82F810B0C2F81CE02A
:10C6900030B115680468A5425AD8651B0560D061A1
:10C6A0004FF0010C52E0029903EB430201EBC2048C
:10C6B00001330599DBB2994208BF0023029911F8B2
:10C6C0003210012947D16268157C002D7FF416AF26
:10C6D000A7685760E76897602769D76064699461C5
:10C6E000049C002CC2D05560C0E7A9EB080424F0DC
:10C6F0007F44BC423ABF3C1B1460C2F800E0C1E773
:10C70000643400206034002061340020583400205C
:10C7100090330020703400204D3400200010014080
:10C720004E34002000E100E0FEFF7F00ED1BE769D2
:10C73000A0463FB13C462768AF42F7D37F1B276036
:10C74000274644461560D761E26102461046D2E6AC
:10C7500080460446EFE70121D0E6FDF741FE24E7DD
:10C76000B5420AD1D269002A7FF450AF08480127A8
:10C77000876091463846BE46B846D5F800B0ED69A8
:10C78000F561002D3FF48DAE2E685E442E6088E684
:10C79000001001402DE9F8432649274B0025C1F838
:10C7A0004051C1F84451C1F84851C1F84C51C1F849
:10C7B0000051C1F804511B68002B39D0D1F8044551
:10C7C0001E49DFF88C800968641A24F07F442F46E4
:10C7D0001A68A24217D8A41A15441A7CDE6982B1DD
:10C7E000D8F800901F74D3E90521B9F1000F06D0E5
:10C7F0001046C84728B1FDF76DFE3346E8E7084606
:10C800009047002EF9D10E4A0E4B11781B788B42BF
:10C8100005D10133DBB2022B08BF0023137012785D
:10C82000094B43F82250094B4FF48012C3F8002102
:10C83000BDE8F8830010014070340020643400200B
:10C8400061340020603400205834002000E100E012
:10C85000603300202DE9FF4700210846FDF7FEFE6A
:10C860004FF0A043B24AB34CC3F82C27B24BB349A4
:10C8700000264FF4AE7220461E7000F0B3F9256812
:10C880006B1C06D032465821201DFDF755FC854211
:10C890000DD04FF4AE720021A648FBF743FE0123F2
:10C8A00000206360FEF706FA08B1FDF713FE43F2BD
:10C8B00008031F682369012B13D063698BB1A56935
:10C8C0009F4E05F6FF7525F47F6525F00F053D4465
:10C8D000B368A52B00F0D58006D8012B13D0002615
:10C8E00063E03D46974EF3E7AA2B00F0D880AC2BCF
:10C8F000F5D12846FEF72AFA002855D131462846B8
:10C90000FEF768FAC9E06369012BE8D1266BD4F819
:10C91000249037444FF0030AA9EB0606B6F5805F72
:10C920004FF000024FF001013846B04628BF4FF4E7
:10C930008058FEF781F80346B0BB42462946384688
:10C94000FEF71CF980BB4FEA98036846CDE900A7C3
:10C9500002950393FDF764FA024628BB012128469D
:10C96000FEF76AF800BB236B43442363FEF7A2F98A
:10C97000B6EB080647444544D0D143F2080332469B
:10C9800018684946FDF7D8FBA36A984204BF012303
:10C99000C4E907036A4808BFC4F81890FDF754FFBC
:10C9A0000020FEF787F900B10126FDF731FE0028CF
:10C9B00040F09680002E00F09A80FDF711FD624B4A
:10C9C000624A1A60624A634F634E052100259170E6
:10C9D000624915805160624A1560624A1570624A68
:10C9E0001570624A4FF48011E020C2F8801182F87D
:10C9F0001403116001F18041A1F56F21F61BC1F80C
:10CA0000085582F811035A4AD1F8041511605949A2
:10CA1000594A0A605949A8320A60594A1570594A58
:10CA20001570594A08211180584A14211180F608BE
:10CA3000AE4275D1564A137843F001031370554B3B
:10CA4000554A1A60554B04221A60554B00221A6051
:10CA5000A36B9BB1FEF70EFC80B1236A002B40F064
:10CA6000A580A369002B00F0A1804E4A13604D4BB6
:10CA70001868FDF7FFFD4C4B01221A70FDF7D4FC3E
:10CA8000FCE72846FEF762F9014600288CD13046C3
:10CA9000FDF7DAFE0846FEF70DF9012683E7314679
:10CAA0002846FEF797F900267DE740F2E730FDF7CC
:10CAB0008DFB15F0030F4FF000010CBF012008465D
:10CAC000FDF7CCFD013DFDF7A3FD60B1002DECD1DC
:10CAD00001210846FDF7C2FD002D7FF46EAF69E726
:10CAE00040F6B835EFE7003518BF0125F0E7FDF750
:10CAF0003FFB00283FF461AF43F208042168FDF7D3
:10CB000091F910B90846FDF7CDF92268FDF78AF9C9
:10CB100010B91046FDF7C6F9002004B0BDE8F08753
:10CB200057F83530984700287FF4BFAE01357FE7CE
:10CB30000C000300AC350020C42E002000F00700DC
:10CB4000D0350020C4350020603300207DB30700BD
:10CB500090330020802C0020882C0020F42D002011
:10CB600070340020603400206134002000E100E0D7
:10CB70006434002014340020A42C00201034002041
:10CB80000C3400201C340020183400201A340020FB
:10CB9000703300205434002065A90700783300204A
:10CBA0007C3300206833002069340020E36A002BC6
:10CBB0007FF464AFA369002B3FF460AF014B626A5E
:10CBC0001A6054E76833002030B501390024A242CE
:10CBD00001D1002005E0035D01340D5DAB42F6D0CC
:10CBE000581B30BD0A44914200F1FF3300D1704719
:10CBF00010B511F8014B03F8014F9142F9D110BD66
:10CC0000F8B500BFF8BC08BC9E467047F8B500BF39
:10CC1000F8BC08BC9E467047002C002050EADA3071
:10CC20008883B89F604F15F30000C98EAF9A070044
:10CC3000539A0700E1990700919C0700779C070031
:10CC4000399C0700F99B070037B20700000000007D
:10CC5000446675546172670008200001FFFFFFFF02
:10CC6000FFFFFFFFFFFFFFFF0000000000000000CC
:10CC70000000000001000000FFFFFFFF512563FCE2
:10CC8000C2CAB9F3849E17A7ADFAE6BCFFFFFFFF47
:10CC9000FFFFFFFF00000000FFFFFFFF96C298D8D4
:10CCA0004539A1F4A033EB2D817D0377F240A463D5
:10CCB000E5E6BCF847422CE1F2D1176BF551BF37DE
:10CCC0006840B6CBCE5E316B5733CE2B169E0F7CB1
:10CCD0004AEBE78E9B7F1AFEE242E34F4B60D2277E
:10CCE0003E3CCE3BF6B053CCB0061D65BC86987674
:10CCF00055BDEBB3E7933AAAD835C65ABF9707009C
:10CD000065970700ED8F0700011101FF010000008A
:10CD100000000000021702FE640000005CCD070066
:10CD2000031704FC04000000FCCD07000000000015
:10CD300000000000000000000101000001000000F0
:10CD400000000000020500002100000000000000BB
:10CD5000000000000000000000000000011104FCC1
:10CD60000400000000000000021104FC04000000A8
:10CD700000000000032104FC040400000000000087
:10CD8000041101FF0100000000000000051102FE77
:10CD90000400000000000000061104FC0400000074
:10CDA00000000000071104FC040000000000000067
:10CDB000081701FF2200000038CD0700091001FF0D
:10CDC00001000000D4CD07000000000000000000BA
:10CDD0000000000000000000011704FC70000000CB
:10CDE00008CD0700021704FCB400000014CE0700B1
:10CDF0000000000000000000000000000101000031
:10CE0000040000000000000000000000000000001E
:10CE100000000000010700007000000008CD0700BE
:10CE200002010000010000000000000003050000F6
:10CE300041000000000000000000000000000000B1
:10CE400000000000982F8A4291443771CFFBC0B593
:10CE5000A5DBB5E95BC25639F111F159A4823F92C5
:10CE6000D55E1CAB98AA07D8015B8312BE8531241E
:10CE7000C37D0C55745DBE72FEB1DE80A706DC9BDF
:10CE800074F19BC1C1699BE48647BEEFC69DC10F8B
:10CE9000CCA10C246F2CE92DAA84744ADCA9B05CC7
:10CEA000DA88F97652513E986DC631A8C82703B08A
:10CEB000C77F59BFF30BE0C64791A7D55163CA0698
:10CEC00067292914850AB72738211B2EFC6D2C4DA4
:10CED000130D385354730A65BB0A6A762EC9C28192
:10CEE000852C7292A1E8BFA24B661AA8708B4BC228
:10CEF000A3516CC719E892D1240699D685350EF452
:10CF000070A06A1016C1A419086C371E4C77482708
:10CF1000B5BCB034B30C1C394AAAD84E4FCA9C5B7E
:10CF2000F36F2E68EE828F746F63A5781478C884CF
:10CF30000802C78CFAFFBE90EB6C50A4F7A3F9BEB1
:10CF4000F27871C6040000040100040220040321E9
:10CF50000404220405230406000407000408000456
:10CF60000900040A00140B00040C00040D00040E58
:10CF700000040F0004100004110004120004130048
:10CF8000041400041500041600041700041800041B
:10CF90001900041A00041B00041C24041D25041E8F
:10CFA00026041F270A00000A01000A02000A0300E3
:10CFB0000A04001A05001A06001A07000A08000AE7
:10CFC00009000A0A000A0B000A0C000A0D000A0EEA
:10CFD000000A0F004901B952C5EF41DE27476A55E3
:10CFE00027B31CE72D1ECB0FA00C3792BE6AB2E907
:10CFF0009B2403956593690B5EF09CFDA5C02CEE08
:10D00000F1ECA5A1470A9B3F814C5FD407D8A3143C
:08D0100004C609D30000000072
:08D0180028B4FF7F01000000B5
:10D020000000000000000000000000000000000000
:10D0300000000000000000000000000000000000F0
:10D0400000000000000000000000000000000000E0
:10D0500000000000000000000000000000000000D0
:10D0600000000000000000000000000000000000C0
:10D0700000000000000000000000000000000000B0
:10D080000090D0030100FFFF258407000184070002
:10D090000010000000300800419E07000000000062
:08D0A000C1B40700B9B3070099
:020000020000FC
:020000041000EA
:041014000080070051
:0410180000E00700ED
:0400000370008539CB
:00000001FF
